gpasm-2.2.29 (Dec 13 2021)   VDCAL_Adjust.asm   2021-12-31  16:42:29         PAGE  1


LOC  OBJECT CODE     LINE SOURCE TEXT
  VALUE

                      00001 #include "mc30p6240.inc"
                      00001                 LIST
                      00002 ;mc30p6240.inc    Standard Header File, Version 1.00 by Sinomcu
                      00367                 LIST
                      00002 
                      00003         org 0x00
                      00004 
0000   2800           00005         goto start
                      00006 
0001                  00007 start:
0001   3C43           00008         bclr    CPPIS
                      00009 
0002   3C88           00010         bclr    CPNIS0
0003   3908           00011         bset    CPNIS1
0004   3D88           00012         bclr    CPNIS2
0005   3A08           00013         bset    CPNIS3
                      00014 
0006   3808           00015         bset            CMPEN
                      00016 
0007   0000           00017         nop
0008   0000           00018         nop
0009   0000           00019         nop
                      00020 
000A   0B00           00021         movai               0x00
000B   15C6           00022         movra               DDR1 
000C   0B00           00023         movai               0x00
000D   1586           00024         movra               P1          
                      00025                 
000E   1589           00026         movra P1KBCR
000F   0000           00027         nop
                      00028 
0010   2800           00029         goto loop
                      00030 
0011                  00031 loop:
                      00032         
0011   0BFF           00033         movai   0xff
0012   1086           00034         XORRA   P1
0013   2800           00035         goto loop
                      00036 
                      00037 
                      00038 
                      00039         en
gpasm-2.2.29 (Dec 13 2021)   VDCAL_Adjust.asm   2021-12-31  16:42:29         PAGE  2


SYMBOL TABLE
  LABEL                             VALUE

CMPCR                             00000043
DDR0                              00000045
DDR1                              00000046
FSR                               00000004
GPR0                              00000007
INDF                              00000000
INTE                              0000000E
INTF                              0000000F
INTF1                             00000044
MCR                               00000008
ODCON                             0000000C
P0                                00000005
P0KBCR                            00000040
P1                                00000006
P1KBCR                            00000009
PCL                               00000002
PCLATH                            0000000A
PUCON                             0000000D
PUDCON                            0000000B
PWMCR0                            00000048
PWMCR1                            00000047
STATUS                            00000003
T0CNT                             00000001
T0CR                              00000041
T1CNT                             0000004D
T1CR                              0000004C
T1DATA                            0000004F
T1DATB                            00000049
T1DATC                            0000004A
T1DATD                            00000042
T1LOAD                            0000004E
TM0CR                             0000004B
_CONFIG0                          00008000
_CONFIG1                          00008001
__1K6240                          00000001
loop                              00000011
start                             00000001
BUZ1EN                            T1CR,5
C                                 STATUS,0
CMPEN                             MCR,0
CMPIE                             CMPCR,2
CMPIF                             INTF1,2
CMPOF                             MCR,5
CPIES                             CMPCR,1
CPNIS0                            MCR,1
CPNIS1                            MCR,2
CPNIS2                            MCR,3
CPNIS3                            MCR,4
CPPIS                             CMPCR,0
DBCLK                             PWMCR0,4
DC                                STATUS,1
DDR00                             DDR0,0
DDR01                             DDR0,1
DDR02                             DDR0,2
DDR03                             DDR0,3
DDR10                             DDR1,0
DDR11                             DDR1,1
DDR12                             DDR1,2
DDR13                             DDR1,3
DDR14                             DDR1,4
DDR15                             DDR1,5
DDR16                             DDR1,6
DDR17                             DDR1,7
EIS                               MCR,6
FSR0                              FSR,0
FSR1                              FSR,1
FSR2                              FSR,2
FSR3                              FSR,3
FSR4                              FSR,4
FSR5                              FSR,5
FSR6                              FSR,6
GIE                               INTE,7
INDF0                             INDF,0
INDF1                             INDF,1
INDF2                             INDF,2
INDF3                             INDF,3
INDF4                             INDF,4
INDF5                             INDF,5
INDF6                             INDF,6
INDF7                             INDF,7
INTIE                             INTE,2
INTIF                             INTF,2
INTM                              T0CR,6
KBIE                              INTE,1
KBIF                              INTF,1
P00D                              P0,0
P00KE                             P0KBCR,0
P00PU                             PUDCON,0
P01D                              P0,1
P01KE                             P0KBCR,1
P01PU                             PUDCON,1
P02D                              P0,2
P02KE                             P0KBCR,2
P02PU                             PUDCON,2
P03D                              P0,3
P03KE                             P0KBCR,3
P03PU                             PUDCON,3
P10D                              P1,0
P10KE                             P1KBCR,0
P10OD                             ODCON,0
P10PD                             PUDCON,4
P10PU                             PUCON,0
P11D                              P1,1
P11KE                             P1KBCR,1
P11OD                             ODCON,1
P11PD                             PUDCON,5
P11PU                             PUCON,1
P12D                              P1,2
P12KE                             P1KBCR,2
P12OD                             ODCON,2
P12PD                             PUDCON,6
P12PU                             PUCON,2
P13D                              P1,3
P13KE                             P1KBCR,3
P13PU                             PUCON,3
P14D                              P1,4
P14KE                             P1KBCR,4
P14OD                             ODCON,4
P14PU                             PUCON,4
P15D                              P1,5
P15KE                             P1KBCR,5
P15OD                             ODCON,5
P15PU                             PUCON,5
P16D                              P1,6
P16KE                             P1KBCR,6
P16OD                             ODCON,6
P16PU                             PUCON,6
P17D                              P1,7
P17KE                             P1KBCR,7
P17OD                             ODCON,7
P17PU                             PUCON,7
PC0                               PCL,0
PC1                               PCL,1
PC2                               PCL,2
PC3                               PCL,3
PC4                               PCL,4
PC5                               PCL,5
PC6                               PCL,6
PC7                               PCL,7
PCH0                              PCLATH,0
PCH1                              PCLATH,1
PD                                STATUS,3
PWM1AEN                           T1CR,6
PWM1AOE                           PWMCR0,7
PWM1AOS                           PWMCR1,7
PWM1BEN                           PWMCR0,1
PWM1BOE                           PWMCR0,6
PWM1CEN                           PWMCR0,0
PWM1COE                           PWMCR0,5
PWM1DEN                           PWMCR1,0
PWM1DOE                           PWMCR1,1
PWM1DOS                           PWMCR1,4
PWM1LG                            PWMCR0,2
PWM1MD                            PWMCR0,3
RST                               STATUS,7
T0CNT0                            T0CNT,0
T0CNT1                            T0CNT,1
T0CNT2                            T0CNT,2
T0CNT3                            T0CNT,3
T0CNT4                            T0CNT,4
T0CNT5                            T0CNT,5
T0CNT6                            T0CNT,6
T0CNT7                            T0CNT,7
T0IE                              INTE,0
T0IF                              INTF,0
T0PRS0                            T0CR,0
T0PRS1                            T0CR,1
T0PRS2                            T0CR,2
T0PTA                             T0CR,3
T0PTS                             T0CR,5
T0SE                              T0CR,4
T0TBS                             TM0CR,7
T1CKS0                            T1CR,3
T1CKS1                            T1CR,4
T1CNT0                            T1CNT,0
T1CNT1                            T1CNT,1
T1CNT2                            T1CNT,2
T1CNT3                            T1CNT,3
T1CNT4                            T1CNT,4
T1CNT5                            T1CNT,5
T1CNT6                            T1CNT,6
T1CNT7                            T1CNT,7
T1DATA0                           T1DATA,0
T1DATA1                           T1DATA,1
T1DATA2                           T1DATA,2
T1DATA3                           T1DATA,3
T1DATA4                           T1DATA,4
T1DATA5                           T1DATA,5
T1DATA6                           T1DATA,6
T1DATA7                           T1DATA,7
T1DATB0                           T1DATB,0
T1DATB1                           T1DATB,1
T1DATB2                           T1DATB,2
T1DATB3                           T1DATB,3
T1DATB4                           T1DATB,4
T1DATB5                           T1DATB,5
T1DATB6                           T1DATB,6
T1DATB7                           T1DATB,7
T1DATC0                           T1DATC,0
T1DATC1                           T1DATC,1
T1DATC2                           T1DATC,2
T1DATC3                           T1DATC,3
T1DATC4                           T1DATC,4
T1DATC5                           T1DATC,5
T1DATC6                           T1DATC,6
T1DATC7                           T1DATC,7
T1DATD0                           T1DATD,0
T1DATD1                           T1DATD,1
T1DATD2                           T1DATD,2
T1DATD3                           T1DATD,3
T1DATD4                           T1DATD,4
T1DATD5                           T1DATD,5
T1DATD6                           T1DATD,6
T1DATD7                           T1DATD,7
T1EN                              T1CR,7
T1IE                              TM0CR,1
T1IF                              TM0CR,0
T1LOAD0                           T1LOAD,0
T1LOAD1                           T1LOAD,1
T1LOAD2                           T1LOAD,2
T1LOAD3                           T1LOAD,3
T1LOAD4                           T1LOAD,4
T1LOAD5                           T1LOAD,5
T1LOAD6                           T1LOAD,6
T1LOAD7                           T1LOAD,7
T1PRS0                            T1CR,0
T1PRS1                            T1CR,1
T1PRS2                            T1CR,2
TO                                STATUS,4
WDTEN                             MCR,7
Z                                 STATUS,2

Errors   :     0
Warnings :     0 reported,     0 suppressed
Messages :     0 reported,     0 suppressed

